:1000000010C028C027C026C025C04DC0B9C022C01E
:1000100021C020C01FC01EC01DC035C11BC01AC0DA
:1000200019C011241FBECFEDCDBF10E0A0E6B0E097
:10003000E0E8F3E002C005900D92A636B107D9F7CB
:1000400010E0A6E6B0E001C01D92A936B107E1F7C5
:1000500071D194C1D5CFD798DF9ABA9AC298D19866
:10006000D998D298DA98D198D9980895F89481B10E
:10007000866081B917B881E086B913B886B1886CFB
:1000800086B978940895F8941FBC8AE08EBD5D9877
:100090001DBC1CBC1BBC1ABC659A61988EB58064E3
:1000A0008EBD789408951F920F920FB60F9211246F
:1000B0002F933F938F939F93F894809167008230A2
:1000C000E9F0833018F4882339F046C0833059F1C1
:1000D000843009F041C02FC024B535B51DBC1CBC0F
:1000E0008EB58F7B8EBD285B3B4029533A4418F474
:1000F000C29A83E011C0C29881E02BC01DBC1CBC19
:10010000C29A8EB58F7B8EBD809166008F5F809383
:100110006600853030F084E08093670010926600BE
:1001200025C083E016C01DBC1CBCC2988EB580647F
:100130008EBD82E00EC01DBC1CBCC2988EB58F7EE9
:100140008EBD6598619A88E592E09BBD8ABD599AFB
:1001500085E0809367000AC0C2981DBC1CBC15BC1A
:1001600014BC8EB580648EBD1092670078949F9108
:100170008F913F912F910F900FBE0F901F90189568
:100180001F920F920FB60F9211248F939F93F894A2
:10019000809167008830B1F1893040F48630D1F029
:1001A000873018F5853009F055C009C08A3009F448
:1001B0003FC08A3080F18B3009F04CC042C0C298F9
:1001C0001DBC1CBC80916000909161009BBD8ABDEC
:1001D00086E008C0C29A1DBC1CBC80E991E09BBDB2
:1001E0008ABD87E08093670046C0C2981DBC1CBCD6
:1001F0008091620090916300885A9D4F9BBD8ABD9B
:1002000088E0F0CFC29A1DBC1CBC80E991E09BBD88
:100210008ABD89E0E7CFC2981DBC1CBC80916400F8
:1002200090916500885A9D4F9BBD8ABD8AE0DACFC8
:10023000C29A1DBC1CBC80E991E09BBD8ABD8BE0CD
:10024000D1CFC2981DBC1CBC8CED95E09BBD8ABD76
:100250008CE0C8CF8EB580648EBD6198659A8EB5EE
:100260008F7E8EBD1DBC1CBC1BBC1ABC15BC14BC37
:10027000109267005D9A78949F918F910F900FBEB6
:100280000F901F9018951F920F920FB60F92112486
:100290002F933F938F939F9386B1877386B924B131
:1002A00035B183E0293E380710F028EE33E087B1FE
:1002B0008C7F87B980916800813031F43093610080
:1002C0002093600082E00DC0823031F430936300EF
:1002D0002093620083E005C03093650020936400A2
:1002E00081E08093680087B190916800892B87B97D
:1002F00086B1886C86B99F918F913F912F910F9015
:100300000FBE0F901F901895809160009091610032
:100310008F5F9F4FC9F380916200909163008F5F60
:100320009F4F91F380916400909165008F5F9F4F84
:1003300059F3089590DEF89481B1866081B917B8B9
:1003400081E086B913B886B1886C86B978948091BB
:100350006000909161008F5F9F4FC9F380916200B0
:10036000909163008F5F9F4F91F380916400909113
:1003700065008F5F9F4F59F386DEFFCFF894FFCF64
:06038000FFFFFFFFFFFF7D
:00000001FF
